:020000040000fa
:080000005e0204000000000094
:020000040000fa
:020000040002f8
:04afe000dfff00008f
:020000040000fa
:020000040002f8
:04afe400ffff00006b
:020000040000fa
:020000040002f8
:04afe80078ff0000ee
:020000040000fa
:020000040002f8
:04afec007dff0000e5
:020000040000fa
:020000040002f8
:04aff00078ff0000e6
:020000040000fa
:1000080000000000000000000000000000000000e8
:100018005602000000000000000000000000000080
:1000280006070000000000000000000000050000b6
:1000380000000000000000000000000000000000b8
:100048002e0500000000000000000000b8050000b8
:100058002406000050060000000000000000000018
:100068000000000000000000000000000000000088
:100078000000000000000000000000000000000078
:100088000000000000000000000000005a05000009
:1000980088050000000000000000000000000000cb
:1000a8000000000000000000000000000000000048
:1000b8000000000000000000000000000000000038
:1000c8000000000000000000000000000000000028
:1000d8000000000000000000000000000000000018
:1000e8000000000000000000000000000000000008
:1000f80000000000000000000000000000000000f8
:1001080000000000000000000000000000000000e7
:1001180000000000000000000000000000000000d7
:1001280000000000f00500000000000000000000d2
:1001380000000000000000000000000000000000b7
:1001480000000000000000000000000000000000a7
:100158000000000000000000000000000000000097
:100168000000000000000000000000000000000087
:100178000000000000000000000000000000000077
:100188000000000000000000000000000000000067
:10019800000000000000000082060000ae0600001b
:1001a800da06000000000000000000000000000067
:1001b8000000000000000000000000000000000037
:1001c8000000000000000000000000000000000027
:1001d8000000000000000000000000000000000017
:1001e8000000000000000000000000000000000007
:1001f80000000000000000000000000000000000f7
:1002080000000000000000000000000000000000e6
:1002180000000000000000000000000000000000d6
:1002280000000000000000000000000000000000c6
:1002380000000000000000000000000000000000b6
:1002480000000000000000000000000000000000a6
:100258000000000000000000000000000000000096
:100268000000000000000000000000000000000086
:0c0278000000000000000000000000007a
:020000040000fa
:10040000803e2000030007008100e900fcff3a0065
:1004100000000600831f7800c20320000400bc0017
:1004200066015100e0815900f23fb1000380b10044
:1004300006003500ee03090000000000423fb10055
:100440000380b100fbff3d001200b000223fb0006e
:10045000020035000280090000000000cf01780092
:1004600000000600861f78006022b8000602200007
:100470000000d0008180d2000482d2008582d200a8
:100480000000a0000202520083825a0003003100e3
:100490000202420083824a000000a1000603e90034
:1004a000f3ff3a004f037800000006000020ef0041
:1004b0000220ef00c088a900004006000f002100c4
:1004c0004032210000018800000000000000eb0025
:1004d000000778000c000900002f78000007eb00ef
:1004e0005420ef000e2eef001e2eef000000eb0058
:1004f00001242100bf1d09008018780040a7a90031
:10050000a1002000beff0700e0022000303a880072
:1005100044e7a90044c7a9004407a9004427a9004b
:100520004447a9004467a9004487a900300020007f
:100530000600fc003174200082072000a30920007f
:10054000824878008348780080487800113a80001b
:10055000618070000600fc0021742000620420000d
:10056000730520008248780083487800804878002e
:100570004427ef00e0022000303a880030002000dd
:100580000d00fc003174200082072000a309200028
:100590008248780083487800804878000000200076
:1005a0002174200062042000730520008248780036
:1005b000834878008048780042a7ae00feff3700ed
:1005c000813e20008eff070010c0b30086e6b70012
:1005d00090c2b300c4e6b70010022000007088008b
:1005e000007825008070880010aea90010cea90008
:1005f000102ea900002ea900100ea90091040700da
:1006000077050700880607008807070035080700f8
:100610004a0807000000eb00817f2100ff0009006d
:10062000805878006e72ef006f72ef006232ef0058
:100630006432ef000080eb00c17e2100050009005c
:10064000801878004a32ef0010cea90014cea9001d
:100650008932a9004c32ef004e32ef005032ef00e9
:10066000262cef00462cef00662cef0000c4b300f0
:1006700084f2b70000c4b30085f2b7005632ef0031
:100680005432ef0010c0b30088f2b7004188a800d0
:1006900041a8a90041c8a80000a1ef0004a1a8003a
:1006a0000481a90005e1a8000068a9002068a8004d
:1006b0001061a8001021a90011e1a80011a1a90052
:1006c00010a1a8001081a8000621ef000821ef006a
:1006d0000ca1ef000ea1ef004408a9004428a900d6
:1006e0004448a9000108a9002108a8001fe1a800aa
:1006f0001fa1a9001ec1a9001ea1a8001e81a8005b
:100700001e61a9001e21a9004d88a8004da8a800bf
:100710004dc8a9001aa1ef000368a9002368a8002a
:1007200021e1a80021a1a90020c1a90020a1a800c1
:100730002081a8002021a9004e08a8004e28a90069
:100740004e48a8000388a90040922000e0088800d5
:100750002388a8002002a9002022a9002042a90085
:1007600020a2a9002062a9002082a90020e2a900fd
:100770002102a9002122a900700720004011880051
:1007800022a2a90022c2a90022e2a90021e2a80017
:100790002182a9004588a90045a8a80045c8a8004d
:1007a0002168a8002828a8000e0ea80021e3a900af
:1007b0002143a80021a3a9002123a9002103a90006
:1007c00020e3a80020c3a80020a3a8002083a9003c
:1007d0002043a90023e3a90023c3a90023a3a90060
:1007e0002343a9002323a9002303a90022c3a900ae
:1007f00022a3a9002283a9002263a9002243a90001
:100800002223a9002203a9002563ef0024e3ef00bf
:100810003223ef002823ef002623ef002e23ef00e2
:100820003023ef0021a8a90001a8a90021e3a90015
:100830004008a9004028a9004048a8002028a90095
:100840000008a900c208a9002bc8a9002be8a9002c
:100850002c08a9000bc8a9000be8a9000c08a900e6
:1008600001eca90001aca900016ca900014ca90090
:10087000012ca900010ca90000eca900008ca90022
:1008800000aca90000cca900000ca900002ca90014
:10089000004ca900006ca900202cef00402cef00b8
:1008a000602cef0004acef00020ca900022ca900a0
:1008b000024ca900262cef00462cef00662cef001e
:1008c000282cef00482cef00682cef000aacef005a
:1008d00023eca80023cca80023aca900238ca900fa
:1008e000236ca900234ca800232ca900230ca900e9
:1008f000222ca90043eca80043cca80043aca900db
:10090000438ca900436ca900434ca800432ca900c8
:10091000430ca90063eca80063cca80063aca90059
:10092000638ca800636ca900634ca800dabc2a00a1
:100930001b32240030002c00fa608800fb60880025
:1009400020618800dabc2a001b32240000402c0001
:10095000fa608800fb60880010618800dabc2a0019
:100960001b32240030002c00fa608800fb608800f5
:1009700020628800dabc2a001b32240000402c00d0
:10098000fa608800fb60880010628800dabc2a00e8
:100990001b32240030002c00fa608800fb608800c5
:1009a00020638800dabc2a001b32240000402c009f
:1009b000fa608800fb60880010638800218ca90021
:1009c000418ca900618ca900216ca900416ca9008f
:1009d000616ca900214ca900414ca900614ca900ff
:1009e00020eca80040eca80060eca8003e2cef0032
:1009f0005e2cef007e2cef0001eca80040013700d8
:100a0000ff3ffc004200f8003600f8004400f80008
:100a10008e1f78000e0020000d000900be1f780018
:100a20003200f8000100fc000068a9000021ef007e
:100a3000ff3ffc003200f900ae0120000d0009006c
:100a40004f1778004f0778004400f9003600f9008e
:100a50004200f9000100fc0000400600ff3ffc00de
:100a60004200f8003600f8004400f8008e1f7800bd
:100a70000e0020000d000900be1f78003200f800b3
:100a80000100fc000108a900ff3ffc003200f90052
:100a9000ae0120000d0009004f1778004f077800c5
:100aa0004400f9003600f9004200f9000100fc00a2
:100ab00000400600ff3ffc004200f8003600f8004e
:100ac0004400f8008e1f78000e0020000d00090081
:100ad000be1f78003200f8000100fc000368a90086
:100ae0001421ef00ff3ffc003200f900ae012000ae
:100af0000d0009004f1778004f0778004400f900f7
:100b00003600f9004200f9000100fc000040060038
:100b1000ff3ffc004200f8003600f8004400f800f7
:100b20008e1f78000e0020000d000900be1f780007
:100b30003200f8000100fc000388a9001821ef0032
:100b40002023a800ff3ffc003200f900ae01200086
:100b50000d0009004f1778004f0778004400f90096
:100b60003600f9004200f9000100fc0000400600d8
:100b7000ff3ffc004200f8003600f8004400f80097
:100b80008e1f78000e0020000d000900be1f7800a7
:100b90003200f8000100fc000168a9006e72ec0050
:100ba0006ed2bf008080fb0030118000827f210068
:100bb00080707900ff3ffc003200f900ae01200098
:100bc0000d0009004f1778004f0778004400f90026
:100bd0003600f9004200f9000100fc000040060068
:100be000ff3ffc004200f8003600f8004400f80027
:100bf0008e1f78000e0020000d000900be1f780037
:100c00003200f8000100fc000828a9002242ae00d2
:100c1000000037002222af002222a900ff3ffc0083
:100c20003200f900ae0120000d0009004f177800d6
:100c30004f0778004400f9003600f9004200f9003f
:100c40000100fc0000400600ff3ffc004200f800ed
:100c50003600f8004400f8008e1f78000e002000d7
:100c60000d000900be1f78003200f8000100fc00f2
:100c70000188a900ff3ffc003200f900ae0120000e
:100c80000d0009004f1778004f0778004400f90065
:100c90003600f9004200f9000100fc0000400600a7
:100ca000ff3ffc004200f8003600f8004400f80066
:100cb0008e1f78000e0020000d000900be1f780076
:100cc0003200f8000100fc0000188000c09288008b
:100cd00001a8a9002003a900ff3ffc003200f90091
:100ce000ae0120000d0009004f1778004f07780073
:100cf0004400f9003600f9004200f9000100fc0050
:100d000000400600ff3ffc004200f8003600f800fb
:100d10004400f8008e1f78000e0020000d0009002e
:100d2000be1f78003200f8000100fc000bc8a900cb
:100d3000ff3ffc003200f900ae0120000d00090069
:100d40004f1778004f0778004400f9003600f9008b
:100d50004200f9000100fc0000400600ff3ffc00db
:100d60004200f8003600f8004400f8008e1f7800ba
:100d70000e0020000d000900be1f78003200f800b0
:100d80000100fc000be8a900ff3ffc003200f90065
:100d9000ae0120000d0009004f1778004f077800c2
:100da0004400f9003600f9004200f9000100fc009f
:100db00000400600ff3ffc004200f8003600f8004b
:100dc0004400f8008e1f78000e0020000d0009007e
:100dd000be1f78003200f8000100fc000c08a900da
:100de000ff3ffc003200f900ae0120000d000900b9
:100df0004f1778004f0778004400f9003600f900db
:100e00004200f9000100fc0000400600ff3ffc002a
:100e10004200f8003600f8004400f8008e1f780009
:100e20000e0020000d000900be1f78003200f800ff
:100e30000100fc000008a9008672ec008612ae00da
:100e400016003700a00880009092880091928000e0
:100e5000700c2000808f500002003e005432ef00e2
:100e60000c00370091928000406e2100808f50006e
:100e7000020036005432ef000600370092928000e4
:100e800003002000b03a29003100200075fd070062
:100e9000a09288001421ef0002003700120eaa0071
:100ea000100ea900ff3ffc003200f900ae01200047
:100eb0000d0009004f1778004f0778004400f90033
:100ec0003600f9004200f9000100fc000040060075
:100ed0006fd2bf006e52e300070032006f72ec0069
:100ee0006fd2bf000080fb00817f210060c07800ce
:100ef00070f2b7000100370070f2ef00000006004a
:100f000030088000109388004008800020938800fb
:100f1000efff070000cfb3007052b50006003900a4
:100f2000e0cfb3007052b500010039000100370076
:100f30007172ef003a01370070f2ae0037003700ef
:100f40007172ef00f0c8b3007052e30005003a0080
:100f500070d2bf0071f2b70072f2ef0073f2ef00cf
:100f60002d003700f0c9b3007052e30005003a00cd
:100f700070d2bf0071f2b70074f2ef0075f2ef00ab
:100f800025003700f0cab3007052e30005003a00b4
:100f900070d2bf0071f2b70076f2ef0077f2ef0087
:100fa0001d003700f0cbb3007052e30005003a009b
:100fb00070d2bf0071f2b70078f2ef0079f2ef0063
:100fc00015003700f0ccb3007052e30004003a0083
:100fd00070d2bf0071f2b7007af2ef000e00370056
:100fe000f0cdb3007052e30004003a0070d2bf00ad
:100ff00071f2b7007bf2ef0007003700f0ceb300cc
:101000007052e30004003a0070d2bf0071f2b700e2
:101010007cf2ef007df2ef00010137007152e20037
:1010200002003a00fe003700fd003700f0c8b300b0
:101030007152e3002f003a0000e0ef007252e3002b
:1010400003003a0070d2bf0072f2b70028003700e8
:1010500070d2bf0073f2b70072d2bf008040780038
:10106000f8cf500007003a004c32ef00262cef007a
:101070008952a900140ea9008072ef008172ef005e
:101080001a00370072d2bf0080407800f9cf5000bc
:1010900007003a005032ef00662cef008972a90079
:1010a000142ea9008272ef008372ef000f00370048
:1010b00072d2bf0080407800fccf500003003a009d
:1010c0004e32ef00462cef000800370030c6b30068
:1010d0007252e30005003a0014cea900f4b7ef0005
:1010e000f6b7ef004a52a9007f12a80072f2ef0093
:1010f000cb003700f0c9b3007152e30088003a001a
:1011000000e0ef007452e30003003a0070d2bf0029
:1011100074f2b7008100370070d2bf0075f2b700db
:101120007552e20026003a0074d2bf008040780079
:10113000f8cf500007003a004c32ef00262cef00a9
:101140008952a900140ea9008072ef008172ef008d
:101150001a00370074d2bf0080407800f9cf5000e9
:1011600007003a005032ef00662cef008972a900a8
:10117000142ea9008272ef008372ef000f00370077
:1011800074d2bf0080407800fccf500003003a00ca
:101190004e32ef00462cef000800370030c6b30097
:1011a0007452e30005003a0014cea9004a52a90087
:1011b000f4b7ef00f6b7ef007f12a8005600370033
:1011c00074d2bf0080407800f8cf500014003a007d
:1011d00075d2bf0091c2b30080cf10000f0036005f
:1011e00020c5b3007552e3000c003e0075d2bf006d
:1011f0000080fb0000004000a163210060807800b7
:101200006092880075d2bf0080f2b70060928000c3
:10121000306188008952a800140ea8003e003700f3
:1012200074d2bf0080407800f9cf500014003a001b
:1012300075d2bf00b1c2b30080cf10000f003600de
:1012400030c5b3007552e3000c003e0075d2bf00fc
:101250000080fb0000004000e16e2100608078000b
:101260008092880075d2bf0082f2b7008092800021
:10127000306388008972a800142ea8002600370069
:1012800074d2bf0080407800fccf500007003a00c5
:1012900075d2bf000080fb004900dd00709288001d
:1012a00070928000306288001b00370030c6b300a7
:1012b0007452e30018003a0014cea80075d2bf00a3
:1012c0008bf2b700f0c7b3007552b5000e003100c5
:1012d0004a52a80075d2bf000080fb000000400009
:1012e000c128210060807800129380002393800041
:1012f00000004100e08049000001be00a2bf88005c
:10130000b3bf8800030037004a52a900f4b7ef00ca
:10131000f6b7ef007f12a80074f2ef00400037002c
:10132000f0cab3007152e3000f003a0000e0ef0092
:101330007652e30003003a0070d2bf0076f2b700a5
:101340000800370070d2bf0077f2b70030c6b30094
:101350007652e30002003a0077d2bf008bf2b7006a
:1013600076f2ef002e003700f0cbb3007152e300ad
:101370000b003a0000e0ef007852e30003003a006f
:1013800070d2bf0078f2b7000400370070d2bf00ff
:1013900079f2b7008100070078f2ef0020003700f3
:1013a000f0ccb3007152e30007003a0000e0ef0018
:1013b0007a52e30003003a0070d2bf007af2b7001d
:1013c0007af2ef0016003700f0cdb3007152e3005f
:1013d00007003a0000e0ef007b52e30003003a0010
:1013e00070d2bf007bf2b7007bf2ef000c00370039
:1013f000f0ceb3007152e30009003a0000e0ef00c4
:101400007c52e30003003a0070d2bf007cf2b700c8
:101410000300370070d2bf007df2b7007cf2ef000e
:101420007f12af004000070030c0b3007e52b5000d
:101430003400310012938000239380005093800089
:1014400061938000800f5100818f59002100390085
:101450006df2a8007e52e20003003a00ec17a800eb
:101460004a12a900060037007ed2bf0080407800f3
:10147000e1cf500002003a00ec37a8004a32a90040
:101480004a52af0004003700f4b7ef00f6b7ef00a0
:1014900014cea9000e00370012ceaa0010cea9006b
:1014a0008bd2bf000080fb0000004000c12821005b
:1014b0006080780012938000239380000000410038
:1014c000e08049000001be00a2bf8800b3bf8800d1
:1014d0001500070065f2ae00090037000621ef0095
:1014e0000821ef006232ef006432ef000080eb0071
:1014f000c17e2100050009008018780080fe3700b9
:101500000400370065f2ae00020037000621ef004c
:101510000821ef006432af0014aea8006432ae00c0
:1015200014aea90076fe37007ef2ef006df2a8003f
:101530004632ef0030928000c200dd00c07e210004
:10154000008040001000be000001be0050938000eb
:1015500061938000800f5100818f59000900310094
:1015600030928000c200dd00c07e2100008040007b
:101570001000be00509388006193880046d2bf00df
:101580007ef2b7004632ec0031928000e38f5000cb
:10159000e8ff3a007f12a9000000060078d2bf00e1
:1015a00080407800f8cf50002f003a0079d2bf0079
:1015b00081f2b7008952ae002a00370020c5b3007f
:1015c0008052b5002700310080d2bf000080fb00b0
:1015d0000006e8000c064600a063210060007e00c3
:1015e0000092880080d2bf000080fb000000400015
:1015f000a1632100608078004012b500f09288005d
:10160000f092800042062000110009000280d800fc
:10161000e0928800e0928000e00f500002003e005f
:1016200010002000e092880081d2bf000080fb0003
:101630005c12bc00e292880080d2bf000080fb00f8
:1016400000004000a16321006080780000928800c3
:10165000e09280004012b4006092880060928000a6
:10166000306188007500370078d2bf008040780074
:10167000f9cf50002f003a0079d2bf0083f2b700b3
:101680008972ae002a00370030c5b3008252b5001f
:101690002700310082d2bf000080fb000006e80076
:1016a0000c064600e06e210060007e00009288007b
:1016b00082d2bf000080fb0000004000e16e2100ec
:1016c000608078004012b50000938800009380008d
:1016d00042062000110009000280d800e092880034
:1016e000e0928000e00f500002003e001000200059
:1016f000e092880083d2bf000080fb005c12bc0037
:10170000e292880082d2bf000080fb00000040000f
:10171000e16e21006080780000928800e0928000f5
:101720004012b4008092880080928000306388006c
:101730004200370020c4b3007852e30029003a0089
:101740007952e20018003a00ecb7ef00eeb7ef0074
:101750004a12a9007f12a800002ea900042ea90099
:101760004c32ef00262cef004e32ef00462cef00fb
:101770005032ef00662cef0010cea90014cea90065
:10178000f4b7ef00f6b7ef004a52a9008172ef00fc
:101790008372ef008952a9008972a900140ea90072
:1017a000142ea9000e003700002ea900042ea80058
:1017b0004c32ef00262cef004e32ef00462cef00ab
:1017c0005032ef00662cef008172ef008372ef0061
:1017d0008952a9008972a900140ea900142ea9002b
:1017e00016003700b0c7b3007852e30013003a0088
:1017f00014cea900f4b7ef00f6b7ef004a52a900e3
:101800004c32ef00262cef004e32ef00462cef005a
:101810005032ef00662cef00ecb7ef00eeb7ef00b0
:101820004a12a9008172ef008372ef008952a90069
:101830008972a900140ea900142ea90078f2ef00f5
:10184000000006008cb3ef00101a2f00709c880077
:1018500010412e00809c880040742d00909c8800d0
:10186000f0b22c00a09c880070fc2b00b09c88007b
:1018700030502b00c09c8800a0ad2a00d09c88006e
:1018800030142a00e09c880060832900f09c8800c6
:10189000b0fa2800009d8800a0792800109d8800db
:1018a000c00020003092880031928000f78f5000f5
:1018b0000e003e00c00020004612b5000006780071
:1018c0000c064600c038210060007e004100de00aa
:1018d000329280004111dd00c13821000101410038
:1018e000000978004632ec00efff3900800120004b
:1018f000309288003192800030022000808f5000aa
:101900000e003e00800120004612b500000678005f
:101910000c064600c038210060007e004200de0058
:10192000329280004111dd00c138210001014100e7
:10193000000978004632ec00eeff3900400220003a
:101940003092880031928000f0022000808f500099
:101950000e003e00400220004612b500000678004e
:101960000c064600c038210060007e004300de0007
:10197000329280004111dd00c13821000101410097
:10198000000978004632ec00eeff39000003200029
:101990003092880031928000b0032000808f500088
:1019a0000e003e00000320004612b500000678003d
:1019b0000c064600c038210060007e004400de00b6
:1019c000329280004111dd00c13821000101410047
:1019d000000978004632ec00eeff3900c003200019
:1019e000309288003192800070042000808f500077
:1019f0000e003e00c00320004612b500000678002d
:101a00000c064600c038210060007e004500de0064
:101a1000329280004111dd00c138210001014100f6
:101a2000000978004632ec00eeff39008004200007
:101a3000309288003192800030052000808f500065
:101a40000e003e00800420004612b500000678001b
:101a50000c064600c038210060007e004600de0013
:101a6000329280004111dd00c138210001014100a6
:101a7000000978004632ec00eeff3900007a2100c0
:101a8000a0a18800f0732100b0a18800f06d2100b2
:101a9000c0a1880000682100d0a188004062210018
:101aa000e0a18800805c2100f0a18800e0562100c0
:101ab00000a288006051210010a28800f04b210094
:101ac00020a288009046210030a2880050412100c9
:101ad00040a28800203c210050a28800103721003d
:101ae00060a288001032210070a28800202d210001
:101af00080a288004028210090a288008023210035
:101b0000a0a28800d01e2100b0a28800301a2100b7
:101b1000c0a28800a0152100d0a2880020112100b9
:101b2000e0a28800c00c2100f0a28800700821000b
:101b300000a388002004210010a38800f0ff2000eb
:101b400020a38800d0fb200030a38800c0f720002d
:101b500040a38800d0f3200050a38800e0ef2000cd
:101b600060a3880000ec200070a3880030e820000b
:101b700080a3880070e4200090a38800c0e02000cb
:101b8000a0a3880020dd2000b0a3880090d9200009
:101b9000c0a3880010d62000d0a38800a0d22000c7
:101ba000e0a3880040cf2000f0a38800e0cb200015
:101bb00000a48800a0c8200010a4880060c52000f0
:101bc00020a4880030c2200030a4880010bf20006c
:101bd00040a4880000bc200050a48800000006003b
:101be0008cb2ef00a0c725007094880050982500a3
:101bf000809488004081250090948800906a250098
:101c0000a094880030542500b0948800303e250010
:101c1000c094880090282500d09488005013250097
:101c2000e094880060fe2400f0948800c0e924005d
:101c30000095880080d524001095880090c124006c
:101c400020958800f0ad240030958800a09a2400eb
:101c500040958800a087240050958800f0742400e7
:101c60006095880090622400709588008050240060
:101c700080958800b03e240090958800302d240087
:101c8000a0958800f01b2400b0958800000b24006c
:101c9000c095880050fa2300d0958800e0e9230021
:101ca000e0958800c0d92300f0958800e0c92300a2
:101cb0000096880040ba230010968800e0aa23000e
:101cc00020968800c09b230030968800e08c23007b
:101cd00040968800307e230050968800d06f230005
:101ce00060968800a061230070968800b05323009e
:101cf00080968800f0452300909688007038230075
:101d0000a0968800202b2300b0968800101e230088
:101d1000c096880040112300d096880090042300cc
:101d2000e096880020f82200f0968800e0eb220080
:101d300000978800d0df220010978800f0d322009f
:101d40002097880050c8220030978800d0bc22001d
:101d50004097880080b122005097880070a622002a
:101d600060978800809b220070978800c0902200b6
:101d7000809788002086220090978800c07b2200f0
:101d8000a097880080712200b097880060672200c9
:101d9000c0978800805d2200d0978800c053220041
:101da000e0978800204a2200f0978800b040220087
:101db000009888006037220010988800402e22008a
:101dc000209888004025220030988800601c22005e
:101dd00040988800b013220050988800200b220001
:101de00060988800b00222007098880060fa210094
:101df0008098880040f221009098880030ea210005
:101e0000a098880050e22100b098880090da210064
:101e1000c0988800e0d22100d098880060cb2100d3
:101e2000e0988800f0c32100f0988800b0bc210041
:101e30000099880080b521001099880080ae2100ab
:101e40002099880090a7210030998800b0a0210037
:101e500040998800009a21005099880060932100e1
:101e600060998800e08c21007099880080862100ac
:101e7000809988003080210090998800007a2100a4
:101e8000a0998800f0732100b0998800f06d2100be
:101e9000c099880000682100d09988004062210024
:101ea000e0998800805c2100f0998800e0562100cc
:101eb000009a880060512100109a8800f04b2100a0
:101ec000209a880090462100309a880050412100d5
:101ed000409a8800203c2100509a88001037210049
:101ee000609a880010322100709a8800202d21000d
:101ef000809a880040282100909a88008023210041
:101f0000a09a8800d01e2100b09a8800301a2100c3
:101f1000c09a8800a0152100d09a880020112100c5
:101f2000e09a8800c00c2100f09a88007008210017
:101f3000009b880020042100109b8800f0ff2000f7
:101f4000209b8800d0fb2000309b8800c0f7200039
:101f5000409b8800d0f32000509b8800e0ef2000d9
:101f6000609b880000ec2000709b880030e8200017
:101f7000809b880070e42000909b8800c0e02000d7
:101f8000a09b880020dd2000b09b880090d9200015
:101f9000c09b880010d62000d09b8800a0d22000d3
:101fa000e09b880040cf2000f09b8800e0cb200021
:101fb000009c8800a0c82000109c880060c52000fc
:101fc000209c880030c22000309c880010bf200078
:101fd000409c880000bc2000509c8800100020001d
:101fe0003092880031928000f0072000808f5000ee
:101ff0000c003e003292800002014100c028210006
:10200000600079004200de00329280004111dd0064
:10201000c128210001014100000978004632ec008e
:10202000f0ff3900000006008000200060a4880056
:102030009000200070a488009000200080a48800f8
:10204000a000200090a48800a0002000a0a4880088
:10205000b0002000b0a48800c0002000c0a4880008
:10206000c0002000d0a48800d0002000e0a4880098
:10207000e0002000f0a48800f000200000a5880007
:10208000f000200010a588000001200020a5880095
:102090001001200030a588002001200040a5880004
:1020a0003001200050a588005001200060a5880064
:1020b0006001200070a588007001200080a58800c4
:1020c0008001200090a58800a0012000a0a5880024
:1020d000c0012000b0a58800d0012000c0a5880064
:1020e000f0012000d0a5880010022000e0a58800a3
:1020f00030022000f0a588005002200000a68800d1
:102100007002200010a688009002200020a68800ff
:10211000c002200030a68800e002200040a688000f
:102120001003200050a688004003200060a688000d
:102130007003200070a68800a003200080a68800fd
:10214000e003200090a6880010042000a0a68800cc
:1021500050042000b0a6880090042000c0a688008b
:10216000e0042000d0a6880020052000e0a688001a
:1021700070052000f0a68800c005200000a7880098
:102180002006200010a788008006200020a78800d5
:10219000e006200030a788005007200040a78800f4
:1021a000b007200050a788003008200060a78800f2
:1021b000b008200070a788003009200080a78800a0
:1021c000c009200090a78800500a2000a0a788001e
:1021d000f00a2000b0a78800900b2000c0a788005c
:1021e000400c2000d0a78800000d2000e0a7880048
:1021f000c00d2000f0a78800900e200000a88800e5
:10220000700f200010a888006010200020a888000f
:102210005011200030a888006012200040a88800db
:102220007013200050a88800a014200060a8880027
:10223000d015200070a888002017200080a88800f2
:102240008018200090a88800f0192000a0a888001d
:10225000801b2000b0a88800201d2000c0a8880096
:10226000e01e2000d0a88800b0202000e0a8880050
:10227000a0222000f0a88800b024200000a9880037
:10228000e026200010a988003029200020a988001d
:10229000a02b200030a98800402e200040a98800f3
:1022a0000031200050a98800f033200060a9880088
:1022b0000037200070a98800403a200080a98800db
:1022c000c03d200090a9880070412000a0a988008e
:1022d00050452000b0a9880070492000c0a988009e
:1022e000d04d2000d0a9880070522000e0a98800bd
:1022f00050572000f0a98800805c200000aa8800c8
:102300000062200010aa8800d067200020aa880060
:10231000006e200030aa88009074200040aa880037
:10232000807b200050aa8800d082200060aa88000c
:10233000908a200070aa8800d092200080aa88008d
:10234000909b200090aa8800d0a42000a0aa88001a
:10235000a0ae2000b0aa880000b92000c0aa880062
:1023600000c42000d0aa8800a0cf2000e0aa8800e6
:1023700000dc2000f0aa880010e9200000ab8800f3
:10238000f0f6200010ab8800a005210020ab8800eb
:102390003015210030ab8800b025210040ab88000b
:1023a0002037210050ab8800a049210060ab880095
:1023b000405d210070ab88000072210080ab880076
:1023c0000088210090ab8800509f2100a0ab8800be
:1023d00000b82100b0ab880030d22100c0ab88002b
:1023e000e0ed2100d0ab8800400b2200e0ab88007c
:1023f000602a2200f0ab8800504b220000ac88001d
:10240000406e220010ac88004093220020ac88006f
:1024100070ba220030ac880000e4220040ac880092
:102420000010230050ac880000000600801c200033
:1024300060ac8800301e200070ac880000202000b6
:1024400080ac8800f021200090ac8800f0232000b0
:10245000a0ac880010262000b0ac880050282000d6
:10246000c0ac8800c02a2000d0ac8800402d2000dd
:10247000e0ac8800f02f2000f0ac8800d0322000c3
:1024800000ad8800d035200010ad88001039200044
:1024900020ad8800703c200030ad88000040200056
:1024a00040ad8800d043200050ad8800e0472000b8
:1024b00060ad8800204c200070ad8800b050200036
:1024c00080ad88007055200090ad8800905a2000a3
:1024d000a0ad8800f05f2000b0ad8800a0652000ae
:1024e000c0ad8800b06b2000d0ad88001072200015
:1024f000e0ad8800e0782000f0ad8800108020007a
:1025000000ae8800a087200010ae8800c08f200099
:1025100020ae88004098200030ae880050a12000f6
:1025200040ae8800f0aa200050ae880010b5200010
:1025300060ae8800e0bf200070ae880040cb200075
:1025400080ae880050d7200090ae880020e42000a4
:10255000a0ae8800b0f12000b0ae880010002100cd
:10256000c0ae8800500f2100d0ae8800701f21003f
:10257000e0ae880090302100f0ae8800a04221003b
:1025800000af8800d055210010af8800306a2100cc
:1025900020af8800b07f210030af880080962100f6
:1025a00040af8800b0ae210050af880050c8210075
:1025b00060af880070e3210070af88003000220017
:1025c00080af8800a01e220090af8800e03e22006d
:1025d000a0af880010612200b0af880050852200b3
:1025e000c0af8800b0ab2200d0af880050d422002a
:1025f000e0af880060ff2200f0af8800002d2300cc
:1026000000b08800605d230010b088009090230027
:1026100020b08800e0c6230030b0880050002400bd
:1026200040b08800403d240050b08800d07d240098
:1026300060b0880020c2240070b08800900a250095
:1026400080b088005057250090b08800a0a82500d1
:10265000a0b08800c0fe2500b0b08800105a260047
:10266000c0b08800c0ba2600d0b088003021270052
:10267000e0b08800b08d2700f0b08800b0002800de
:1026800000b18800807a280010b1880090fb2800f3
:1026900020b188005084290030b1880030152a000c
:1026a00040b18800b0ae2a0050b1880040512b00e4
:1026b00060b1880090fd2b0070b1880010b42c0030
:1026c00080b1880070752d0090b1880050422e00b6
:1026d000a0b18800601b2f00b0b1880038b6ef00b1
:1026e0000000060010002000309288003192800027
:1026f00020052000808f50000d003e0032928000a7
:1027000002014100c04821006000790062042000fd
:102710000200b800329280004111dd00a163210067
:1027200001014100000978004632ec00efff39005a
:10273000b0f92f0000b788000000060050ad22005d
:10274000f0ba880040c9220000bb880040ee220099
:1027500010bb8800c01c230020bb880080432300de
:1027600030bb8800c064230040bb8800c0872300c2
:1027700050bb880040c6230060bb8800c0fa23001d
:1027800070bb8800002d240080bb8800408324009b
:1027900090bb880080d32400a0bb88004026250081
:1027a000b0bb880080902500c0bb880080fa25005f
:1027b000d0bb8800807a2600e0bb88000007270095
:1027c000f0bb880080b1270000bc88008071280021
:1027d00010bc88004032290020bc8800c0df2900de
:1027e00030bc8800c07f2a0040bc8800801b2b00c2
:1027f00050bc880080d72b0060bc880080972c00dc
:1028000070bc880000762d0080bc880080582e00a7
:1028100090bc8800406c2f00a0bc8800c002200043
:10282000309288003192800070032000808f500029
:102830000e003e00c00020004612b40000067800e2
:102840000c064600e06e210060007e004100de00c4
:10285000329280004111dd00e16e21000101410052
:10286000000978004632ec00eeff390040052000f8
:102870003092880031928000f0072000808f500055
:1028800008003e00329280004111dd00e16e21001f
:1028900001014100406c2f00000978004632ec0035
:0c28a000f4ff390000000600ffff3700c5
:020000040000fa
:1028ac0040120000060000008000000046120000ec
:1028bc001c00000080000000621200000c000000f0
:1028cc00800000006e1200001e000000800000005e
:1028dc008c1200006005000080000000ec17000066
:1028ec000c00000080000000f81700000001000040
:0828fc00800000000000000054
:00000001FF
